:1000000083161C308500003086008312A8288207E2
:100010003E34413441343E34003420347F340034A3
:10002000273449344934313422344934493436345C
:100030001C3424347F3404347A344934493446340B
:100040003E344934493426344034473448347034DB
:1000500036344934493436343234493449343E3400
:1000600000348514000085101708A30004309800A0
:100070002308072086005520A30A980B3828003053
:10008000950055200800851400008510003086007A
:1000900055201908A4000430980024080720860081
:1000A0005520A40A980B4D2808009B0B55280030BA
:1000B0008600051000000514080004309B009A0B10
:1000C0005F289B0B5F280800A20A990A990A990ADF
:1000D000990AA21C0800A21D08000030A200990085
:1000E000A10A970A970A970A970AA11C0800A11D5E
:1000F00008000030A10097000800A20399039903AB
:1001000099039903221E08000930A20024309900A7
:10011000A1039703970397039703211E0800093053
:10012000A100243097000800051D97289C289E1ADE
:1001300008009E16642008009E120800051EA128D3
:10014000A6281E1B08001E177D2008001E1308008D
:100150000030A100A2009700990060309C0031207F
:1001600094209E209C0BAF2810309C005D20942092
:100170009E209C0BB62860309C00432094209E203B
:100180009C0BBD28A0309C005D2094209E209C0BE1
:04019000C428AD28AA
:00000001FF
